:1000000001308A00E1290000D3346D38EC32202A17
:10001000E832F236EF36653AE8327210A0060A008E
:10002000533A613B3A10253220147039EF3165376D
:10003000F430A9060A00533A613B3A1025322014E5
:100040007039EF316537F430A9060A00533A613B45
:100050003A10253275147039EF316537F430A9063E
:100060000A0083168611831286110830F80038289A
:100070000000F8174928F813AB0C03188615031C69
:100080008611781749287813F80B3C284728000078
:1000900086153F308400840B4B280000F81B3B285A
:1000A000781B43280800831603178C170C140000D4
:1000B000000083120C087F39031997280313A4004A
:1000C00003170D080313A50003170F080313A60059
:1000D0002408AB003120250803178D0003132608E0
:1000E00003178F0083168C170C1400000000831276
:1000F0000C0D0E0D7F39031997280313A400031765
:100100000D080313A50003170F080313A600240806
:10011000AB003120250803178D00031326080317B1
:100120008F008D0A03198F0A031353280317031333
:100130008A110A12492A0830F80000008610831636
:10014000861000008312A40D0610031CAA28831633
:10015000061483120318AF28831606108312831621
:1001600086148312861CB228F80B9D280000861086
:100170008316861000000614000000008614831207
:10018000861CC028F8010000061878148610831613
:10019000861083120610831606108312080008309A
:1001A000A5007708A60083160614000086148312A3
:1001B000861CD82806180314061C0310F80D00002E
:1001C0008316861083128610A50BD3288316061477
:1001D00000008312061026080319F1288316061062
:1001E00083120000831686148312861CF5280000F3
:1001F00086108316861000008312061083160610E0
:1002000083120800831603178C170C1400000000DB
:100210000318312983120C087F390313A600031732
:100220000D080313A70003170F080313A8002608DF
:10023000AB003120270803178D000313280803178C
:100240008F0083168C170C14000000008312031318
:10025000A50B2B292E298316031731295029831624
:10026000031783120C0D0E0D7F390313A60003171D
:100270000D080313A70003170F080313A80026088F
:10028000AB003120270803178D000313280803173C
:100290008F008D0A03198F0A03100313A50B02297F
:1002A00008002C08F8012B02031859292B08F70025
:1002B0006529F7010830AD00AB0DF70D2C0877026A
:1002C0000318F700F80DAD0B5C2908002030261E3E
:1002D0003030A7002508F700A51F7529F709F70A90
:1002E0007708A5002D30A700A6172508AB006430BD
:1002F000AC0051217708A50030307807A800250808
:10030000AB000A30AC00512130307707AA00303002
:100310007807A9002708F700A61D9029A61F261117
:10032000261A9D29A61FB8292619B8297708A800DA
:10033000A618B8297708A900B82930302802031D6B
:10034000B8297708A8002030A700A61DAB292611E0
:10035000A614A61FA61030302902031DB82977085D
:10036000A9002030A800A61DAB29A610A61F2610A4
:10037000261DBD292708AB003120A61CC22928084C
:10038000AB003120261CC7292908AB0031202A08E0
:10039000AB003120080025308400831300080319C6
:1003A000DE290230F800F701F70BD429F80BD32926
:1003B0009730F700F70BDA29800BD1298A110A123E
:1003C000572B840183131F308305713083168F00F0
:1003D0000F08861183128615831603170908C03982
:1003E000890003131F129F12003003178800831225
:1003F000870188018901FF300313A00083160317CA
:100400000908C039890003131F129F120030031717
:100410008800831203131F139F1383169F138312E5
:100420001F149412A012200883168700831220162E
:100430002008831687008312A011200883168700E6
:100440000130831294000030831694000108C739EC
:1004500008388100831290010030F80092000030CB
:1004600083169200831220152008831687008312BA
:10047000970183169B019C0101309D008312031795
:1004800087018801890104308D0000308F0003133B
:1004900053288316061400008614000083120610E9
:1004A0008316061000008312861083168610D13042
:1004B0008312A4009B207808231078182314831635
:1004C0000610000086148312861C642A0000682A25
:1004D000000083160614000001308312A306831661
:1004E0000610000086148312861C742A0000782AE5
:1004F0000000831606140000061400008614000095
:1005000083120610831606100000831286108316CD
:100510008610D0308312A4009B202830A4009B209A
:1005200083160610000086148312861C952A00008C
:10053000992A000083160614000006140000861491
:100540000000831206108316061000008312861026
:1005500083168610D1308312A4009B20F701CF2090
:100560007808A10083160610000086148312861CEA
:10057000B72A0000BB2A00008316061400000614E8
:100580000000861400008312061083160610000077
:100590008312861083168610D0308312A4009B200D
:1005A0000F30A4009B2083160610000086148312CF
:1005B000861CD82A0000DC2A0000831606140000DE
:1005C000061400008614000083120610831606101D
:1005D00000008312861083168610D1308312A40087
:1005E0009B20F701CF207808A20083160610000098
:1005F00086148312861CFA2A0000FE2A0000831645
:10060000061400000030831223180130A4001030BB
:1006100003178D0000308F00031006300313A50070
:1006200002212408A5001F30A600662114300317FC
:100630008D0000308F0003100D300313A500022140
:100640001B3003178D0000308F000310063003139A
:10065000A50002212108A5001F30A60066211F3039
:1006600003178D0000308F0003100D300313A50019
:100670000221263003178D0000308F000310063052
:100680000313A50002212208A5001F30A600662141
:100690002A3003178D0000308F0003100D30031334
:1006A000A50002210830A400FA30A500CB29A40B34
:0606B000542B492A6300EF
:04400E00F52CFF3F4F
:00000001FF
